:1000000022C03CC03BC03AC039C038C037C036C03F
:1000100035C034C033C032C031C030C02FC02EC054
:100020002DC02CC02BC02AC029C028C027C026C084
:1000300025C024C013C517C50CC506C500C552C5CB
:100040006FC58BC5A0C511241FBECFEFD4E0DEBFA6
:10005000CDBF11E0A0E0B1E0EEEDF1E102C005900E
:100060000D92A63EB107D9F712E0A6EEB1E001C0AD
:100070001D92AA30B107E1F760D1AFC8C1CF9C0192
:10008000F999FECF32BD21BDF89A80B508959C0143
:10009000F999FECF1FBA32BD21BD60BD0FB6F894ED
:1000A000FA9AF99A0FBE089583E080937C0086E067
:1000B00080937A0080917A00806880937A008091A2
:1000C0007A00806480937A0080917A0086FDFCCF6C
:1000D00080917800909179000895EAE7F0E08081BE
:1000E0008F77808308956295660F660F607C8F71AD
:1000F000862B80937C008AEF90E00197F1F7809146
:100100007A00806480937A0080917A0086FDFCCF2B
:100110002091780030917900C90108950F931F93C1
:10012000082F482F4F71406C40937C008AEF90E07D
:100130000197F1F780917A00806480937A00809132
:100140007A0086FDFCCFE0917800F0917900409331
:100150007C008AEF90E00197F1F780917A0080644B
:1001600080937A0080917A0086FDFCCF2091780000
:100170003091790040937C008AEF90E00197F1F78D
:1001800080917A00806480937A0080917A0086FD65
:10019000FCCF609178007091790040937C008AEFE9
:1001A00090E00197F1F780917A00806480937A0063
:1001B00080917A0086FDFCCF809178009091790043
:1001C0002E0F3F1F260F371F280F391F10E0000F7B
:1001D000111FF801EE50FE4F31832083F801EA51E0
:1001E000FE4F6081718180E090E040E050E099D75F
:1001F0009B01AC019A0144275527F801E556FE4FB3
:1002000080819181AA2797FDA095BA2F280F391FC9
:100210004A1F5B1F02501E4FF80131832083C90122
:100220001F910F9108958EE480937C008AEF90E0F7
:100230000197F1F780917A00806480937A00809131
:100240007A0086FDFCCF809178009091790084EC53
:1002500099E00197F1F78EE480937C008AEF90E0BB
:100260000197F1F780917A00806480937A00809101
:100270007A0086FDFCCF209178003091790080ECE7
:1002800080937C008AEF90E00197F1F780917A00EB
:10029000806480937A0080917A0086FDFCCF809103
:1002A00078009091790084EC99E00197F1F740E0B3
:1002B00050E06CE273EB81E090E052D7C901089501
:1002C000982F662319F08BB1892B03C08BB19095C1
:1002D00089238BB908958AB187608AB98BB1876009
:1002E0008BB9089580917A008F7780937A00EBD64E
:1002F00083B7817F846083BF83B7816083BF889524
:1003000083B78E7F83BFD1D583E080937C0086E066
:1003100080937A0080917A00806880937A0080913F
:100320007A00806480937A0080917A0086FDFCCF09
:10033000809178009091790008952F923F924F928A
:100340005F926F927F928F929F92AF92BF92CF9265
:10035000DF92EF92FF920F931F93DF93CF93CDB76E
:10036000DEB764970FB6F894DEBF0FBECDBF8AB17B
:1003700087608AB98BB187608BB98BB188638BB981
:100380008AB1877C8AB9569A82E484BD82E085BDB1
:1003900080917E008F6380937E0087D583E0809379
:1003A0007C0086E080937A0080917A008068809358
:1003B0007A0080917A00806480937A0080917A003C
:1003C00086FDFCCF809178009091790067D5F999EE
:1003D000FECF83E090E092BD81BDF89A20B423E087
:1003E000221508F42224F999FECF81E090E092BD15
:1003F00081BDF89A30B43FE0331510F415E0312E8A
:10040000E32DF0E0EB53FE4F808187BDF999FECFDD
:1004100082E090E092BD81BDF89A80B5F999FECF57
:1004200084E090E092BD81BDF89AB0B4F999FECF16
:1004300085E090E092BD81BDF89A40B5498B842F4C
:100440008251823510F05CE1598B86E090E06FE3D9
:1004500070E03CD63C016FE78F3F960710F06624B2
:100460007724B6EEEB2EB1E0FB2E08E010E0A8E812
:10047000CA2EA8ECDA2EC8016FE370E027D6F70188
:100480009183808380549C498F5B934618F0F701D9
:10049000D182C0820C5F1F4F22E030E0E20EF31EDB
:1004A0000032110541F7BFDE9E878D8710E0812F56
:1004B00035DE1F5F1630D9F7BA8ABB2011F031E064
:1004C0003A8B8AE05989589FA0011124588B4F8795
:1004D000DE011196E5EDF1E089E001900D92815089
:1004E000E1F78BB1887F8BB9A22C8824992444240E
:1004F00055241C8A1B8A1FEFCC24DD24BB241C86B8
:100500001B861A86880C991C89B190E0E3E09695C9
:100510008795EA95E1F721E030E082279327817003
:100520009070882A992A440C551C89B190E064E0A7
:10053000969587956A95E1F7822793278170907049
:10054000482A592A6B897C89660F771F89B190E008
:1005500045E0969587954A95E1F782279327817024
:100560009070682B792B7C8B6B8B7FEF87167FEFDE
:10057000970661F48FEF48168FEF580639F499E02B
:10058000A92ECC24DD2491E09C871B8681E0E82EF7
:10059000F12CE820F92080FE09C080E0EFEF8E16F4
:1005A00009F481E0882311F4589A01C0589840FE5C
:1005B00002C0599A01C05998FB89F0FF02C05A9AAB
:1005C00001C05A98A21469F022E02A1550F439E5C6
:1005D000C31632E0D30628F061D4A22CCC24DD244B
:1005E000BB24C60193708050934051F41CDE9E875B
:1005F0008D876F8578898617970710F403E0A02E02
:100600007A89772389F080E3C81685E7D80660F4F5
:1006100080E090E0ED85FE852F8538892E173F0715
:1006200028F481E090E002C080E090E046D531E619
:10063000C3163AEED30610F055DEAA244C854423A7
:1006400041F0EF2869F540FC2BC05B8951705C8755
:1006500029C06FEF861661F4A39473E07A1508F44D
:10066000AA241CD4BB2481E08C8792E09B871FC006
:10067000C40187789070069729F488249924E1E0D2
:10068000EB8715C0C20187709070069711F4F4E0F3
:10069000C5C38B899C8987709070069731F4BDC360
:1006A00021E02C873B85332311F41B8602C0CC2428
:1006B000DD2442E0A41609F448C14A1538F0AA2006
:1006C00071F051E0A51609F09FC3EAC063E0A616D9
:1006D00009F48FC179E0A71609F096C3C4C21123AB
:1006E00011F08CE0BCD380E019DD9093FF01809382
:1006F000FE0181E013DD909301028093000282E00D
:100700000DDDAC01909303028093020285E04C3D25
:1007100058071CF4E1E0F0E021C08091FE019091C7
:10072000FF01E1E0843F9E079CF0209100023091A0
:100730000102B901681B790BCB01845F914044F041
:10074000E0E0F0E0CA01821B930B845F914014F457
:10075000E1E0F0E039E041365307DCF48091FE013E
:100760009091FF0163E0813296079CF42091000292
:1007700030910102B901681B790BCB018152934082
:1007800044F460E070E0CA01821B930B81529340F5
:1007900014F061E070E089B18873883309F03EC0DD
:1007A0003E2FEE2339F0C60187709070892B11F42B
:1007B0005A9A01C05A98262F662339F0C6018770CD
:1007C0009070892B11F4599A01C05998222329F568
:1007D000332319F536E0453A5307FCF08091FE01CA
:1007E0009091FF0162E087329607BCF020910002F1
:1007F00030910102F901E81BF90BCF0187529240B9
:1008000064F0421B530B475252403CF0C6018F73B9
:100810009070892B11F4589A01C05898C6018F70B6
:100820009070892B09F0F0C280E061E087D3C301AA
:1008300065E040E0A4D380E091E095D3809102028E
:100840009091030265E042E09AD380E062E076D3C3
:100850008091FE019091FF0164E042E090D385E039
:1008600062E06CD380910002909101022091FE0120
:100870003091FF01821B930B65E042E0ECD38BE0EB
:1008800062E05CD380910202909103022091000209
:1008900030910102821B930B65E042E0DCD3B4C2CD
:1008A000113029F08CE0DBD28BB1887F8BB9C60187
:1008B0008F709070892B09F0A7C280E061E03ED371
:1008C00087E091E050D3AFDC9E878D8764E042E003
:1008D00056D38CE091E047D380917B0190917C01CD
:1008E0000B9641D34D855E856F85788946175707EE
:1008F00078F480E062E022D380E191E034D380E2BA
:100900009EE4E9E1F0E03197F1F70197D1F7EADCF5
:1009100085E004DC80E062E011D380E291E023D343
:10092000809108029091090265E041E094D383E24E
:1009300091E019D38091FC019091FD0164E040E0C9
:100940001ED388E291E00FD35FC2C6018F70907012
:10095000892B09F059C2123029F08CE080D28BB17A
:10096000887F8BB980E0DADB9093FF018093FE01F2
:1009700081E0D4DB909301028093000282E0CEDB21
:10098000909303028093020283E0C8DB90930502F8
:100990008093040280E061E0D1D28AE291E0E3D268
:1009A0008091FE019091FF0165E042E0E8D28DE286
:1009B00091E0D9D2809100029091010265E042E07D
:1009C000DED280E062E0BAD281E391E0CCD28091C5
:1009D00002029091030265E042E0D1D284E391E00B
:1009E000C2D2809104029091050265E042E0C7D234
:1009F0000BC2133029F08DE032D28BB1887F8BB9D6
:100A00007B85713051F4B39488E08B1508F4BB24D6
:100A100080E593EC0197F1F7E4C09B85692F70E0C6
:100A2000CB0184719070892B09F4D5C0EB2DF0E0D7
:100A3000E930F10508F0D5C0E65EFF4F099480E08B
:100A400090E0A0E0B0E01EC080E090E0A0E0B0E068
:100A500016C080E090E0A0E0B0E00DC088E293E234
:100A6000A0E0B0E004C080E090E0A0E0B0E08C57EF
:100A70009C4FAF4FBF4F865A9F4FAF4FBF4F099606
:100A8000A11DB11D7C018D010894E11CF11C011D0B
:100A9000111D62FF12C08FEF9FE7A0E0B0E08E193A
:100AA0009F09A00BB10B930140E050E028173907D4
:100AB0004A075B0710F46E0C7F1C64FF0CC0C30177
:100AC000A0E0B0E0E816F9060A071B0710F4D80109
:100AD000C701681A790A86E090E0B30147E450E064
:100AE0000BD37FC062FF05C03394E0E13E1609F4EA
:100AF000332464FF06C03A94FFE0F31510F4BFE01E
:100B00003B2EE32DF0E0EB53FE4F808187BDF9993A
:100B1000FECF1FBA81E090E092BD81BD30BC17C00E
:100B200062FF05C0239424E0221609F4222464FF06
:100B300006C02A9433E0321510F4A3E02A2EF99966
:100B4000FECF1FBA83E090E092BD81BD20BC0FB6FE
:100B5000F894FA9AF99A0FBE44C020E04A894423D7
:100B600009F421E02A8BF999FECF1FBA84E090E0C6
:100B700092BD81BD20BD0FB6F894FA9AF99A0FBEC6
:100B8000822F9BD22EC062FF07C059895F5F598BAD
:100B9000513310F082E1898B64FF07C0998991502D
:100BA000998B923110F4E0E3E98BF999FECF1FBAEB
:100BB00085E090E092BD81BDF989F0BD0FB6F89453
:100BC000FA9AF99A0FBE8AE03989389F9001112468
:100BD000388B2F8706C0C6018F709070892B09F063
:100BE00013C180E061E0AAD188E391E0BCD1C301E8
:100BF00065E040E0C4D182E491E0B5D180E062E0FC
:100C00009DD185E491E0AFD149E0431510F080E338
:100C100001C087E5830D04D187E491E0A4D1822D42
:100C200090E061E040E0ABD18AE491E09CD18A8918
:100C300090E061E040E0A3D18DE491E094D1898916
:100C400090E063E041E09BD180E591E08CD1E1E070
:100C5000F0E0EC0FFD1FEB0DF11D6081862F8F7012
:100C600062956F70D0C0193029F08DE0F8D08BB14B
:100C7000887F8BB95B855130B1F56A85662361F158
:100C80000B2D10E0000F111FF801E250FE4FD801AC
:100C9000A556BE4F608171812D913C91621B730BF3
:100CA000882777FD8095982FCB0177276627F80155
:100CB000EE50FE4F2081318140E050E073D2F801C8
:100CC000EA51FE4F31832083000F111FC80108969F
:100CD000B90147E450E010D2B39475E07B1508F4F5
:100CE000BB241A865FC08B85482F50E0CA018471EF
:100CF0009070892B09F44EC0C20183709070892BCB
:100D0000A9F08B899C8983709070892B79F0EB2DE9
:100D1000F0E0EE0FFF1FEA51FE4F88E898EC918358
:100D200080838B2DFBD991E09A873CC042FF18C08D
:100D3000EB2DF0E0EE0FFF1FDF01A250BE4F2D9113
:100D40003C911197ED54FE4F80819181281739070E
:100D50003CF42F5F3F4F2D933C93E1E0EA8722C0A4
:100D600044FF1EC0EB2DF0E0EE0FFF1FDF01A2508D
:100D7000BE4F2D913C911197E955FE4F8081918195
:100D8000821793076CF4215030402D933C93F1E08F
:100D9000FA8708C0C6018F709070892BA9F502C030
:100DA00021E02A8780E061E0C9D082E591E0DBD0D4
:100DB00080E062E0C3D00B2D10E07801EE0CFF1C48
:100DC000F701E157FE4F80819181CDD083E691E01C
:100DD000CAD0F701E250FE4F01541E4F808191812D
:100DE00065E0F801408137D185E691E0BCD026EE80
:100DF00031E0E20EF31EF7018081918165E040E071
:100E0000BED086E062E09AD084ED90E30197F1F7DE
:100E10000894C11CD11C1A2D75CBF0E1FB8747CC7F
:100E20002D9A95B1907F95B925B1982F92959F7085
:100E3000922B95B92C9A21E0922F9A95F1F72C9844
:100E400095B1907F95B995B18F70982B95B92C9AE3
:100E50002A95F1F72C9888E38A95F1F708952D9853
:100E600095B1907F95B925B1982F92959F70922B4F
:100E700095B92C9A21E0922F9A95F1F72C9895B17B
:100E8000907F95B995B18F70982B95B92C9A2A952A
:100E9000F1F72C9883E38A95F1F7089581E0DFDF7D
:100EA00083E397E00197F1F7089584B18FEF84B958
:100EB00085B1807C85B985B1806C85B980E096E389
:100EC0000197F1F785B1807F85B985B1836085B9D8
:100ED0002C9A21E0822F8A95F1F72C9840E052E17C
:100EE000CA010197F1F72C9A822F8A95F1F72C9875
:100EF00089E993E0FC013197F1F72C9A322F3A956A
:100F0000F1F72C980197F1F785B1807F85B9299A7F
:100F10002C9A2A95F1F72C98CA010197F1F788E2EB
:100F20009EDF8CE09CDF86E09ADFB8DF089582E0E8
:100F300096DF83E397E00197F1F70895623061F05F
:100F4000633018F4613071F405C0633039F06430F7
:100F500049F406C0805805C0805403C0805701C0C2
:100F600080537DDF0895CF93DF93EC0102C021967B
:100F700057DF88818823D9F7DF91CF9108957F9239
:100F80008F929F92AF92BF92CF92DF92EF92FF9299
:100F90000F931F93DF93CF93CDB7DEB728970FB68C
:100FA000F894DEBF0FBECDBF9C01DE011196EEEDC1
:100FB000F1E088E001900D928150E1F7411161501C
:100FC000762E7A94790194E0D92ECC24C3944E01E4
:100FD0000894811C911CA42EBB24DA940D2D10E0E2
:100FE000F801EE0FFF1FE80DF91D0190F081E02DD3
:100FF00080E3222733272E1B3F0B04C08F5FE20EB6
:10100000F31ECC24EE16FF06C8F7D71418F4C1104F
:1010100080E206DF0F5F1F4FA016B10619F48EE2C3
:10102000FFDECC24DD20C9F68E2D805DF9DE28960A
:101030000FB6F894DEBF0FBECDBFCF91DF911F91E9
:101040000F91FF90EF90DF90CF90BF90AF909F9067
:101050008F907F9008950F931F93CF93DF93EC01B0
:10106000162F042F97FF06C0D095C195DF4F8DE254
:10107000D7DE1150CE01612F402F81DFDF91CF915C
:101080001F910F9108950F931F93CF93DF938B01BF
:10109000880F880F880F8064E2DEC0E0D0E0F8019E
:1010A000EC0FFD1F8081BCDE2196C830D105B9F759
:1010B000DF91CF911F910F910895882311F02E9AFF
:1010C00008952E98089585B115B80895DF92EF928E
:1010D000FF920F931F937B018C01FB010995D82E82
:1010E000C8010196F7010995982F8D2D1F910F9139
:1010F000FF90EF90DF900895DF92EF92FF920F93B1
:101100001F93D72E7A018C01FA010995C801019627
:101110006D2DF70109951F910F91FF90EF90DF90D2
:101120000895629FD001739FF001829FE00DF11D31
:10113000649FE00DF11D929FF00D839FF00D749F51
:10114000F00D659FF00D9927729FB00DE11DF91FFD
:10115000639FB00DE11DF91FBD01CF01112408955A
:10116000A1E21A2EAA1BBB1BFD010DC0AA1FBB1FAB
:10117000EE1FFF1FA217B307E407F50720F0A21B1D
:10118000B30BE40BF50B661F771F881F991F1A948A
:1011900069F760957095809590959B01AC01BD01B4
:1011A000CF01089597FB092E05260ED057FD04D0D8
:1011B000D7DF0AD0001C38F4509540953095219522
:1011C0003F4F4F4F5F4F0895F6F79095809570957C
:0E11D00061957F4F8F4F9F4F0895F894FFCF8A
:1011DE004B4D2020553D005663633D005620560072
:1011EE00556E7465727370616E6E756E6721210037
:1011FE00543D00DF432028002900313A0020323AC6
:10120E0000333A0020343A004C2E4C6164756E6700
:10121E003A004B4D004B00204D00204C0020550055
:10122E00560021214B616C696272696572756E6739
:10123E002121003D00204B3D0024526576697369E3
:10124E006F6E3A20312E313920240069015531005C
:10125E005532005533005534005430005431007D62
:10126E000180018301860189018C010000000000CC
:10127E0000000055F555F50000000000000000D4F8
:10128E00FED4FEB80BB80BB80BB80BF401F4010288
:10129E00020202010101020305080C11171E262F7E
:1012AE003944505D6B191A1B1C1D2124272C0A0072
:0612BE006400E8031027A4
:00000001FF
